:0400000000000000FC
:0400010000000000FB
:0400020000000000FA
:040003002150000F79
:040004003AECF03DA5
:04000500370400B705
:0400060011E660019E
:04000700108216212C
:040008002150000F74
:040009001128103D6D
:04000A001904014F85
:04000B0000000000F1
:04000C0000000000F0
:04000D0000000000EF
:04000E002150000F6E
:04000F0031ECF07D63
:040010003F04021790
:0400110011E6600193
:040012001082162121
:040013002150000F69
:040014001A28107D19
:04001500170402AF1B
:0400160000000000E6
:040100000FC6000C1A
:040101003B7A07C17D
:040102000CA41660D3
:04010300240424317B
:040104003BC6100FD7
:040105002BC60240C3
:040106002FD20001F3
:0401070014F20001ED
:0401080012C20038E7
:040109002FD20001F0
:04010A0014F20001EA
:04010B0038B2D00036
:04010C00358210190F
:04010D0000000000EE
:04010E0000000000ED
:04010F0000000000EC
:0401100000000000EB
:0401110000000000EA
:0401120000000000E9
:0401130000000000E8
:0401140000000000E7
:0401150000000000E6
:0401160000000000E5
:0401170000000000E4
:0401180000000000E3
:0401190000000000E2
:04011A0000000000E1
:04011B0000000000E0
:04011C0000000000DF
:04011D0000000000DE
:04011E0000000000DD
:04011F00020423EFC4
:0401200000000000DB
:0401210013C20710EE
:040122000B88C20084
:04012300030421A10F
:0401240004C60020ED
:040125003B280C085F
:040126003EC6C80009
:04012700162002019B
:040128001420C200DD
:04012900070421AFF7
:04012A0000000000D1
:0402000024B2562DA1
:0402010019AE01AD84
:0402020034C60FF1FE
:0402030000C61FF220
:040204002550000180
:0402050007C7FFF335
:040206001AB1B3C0B6
:0402070017044B107D
:040208000FB1C3C0AF
:040209001F044E3050
:04020A0020C9001FE8
:04020B0034044B115B
:04020C000183152F26
:04020D001D833561B7
:04020E003E90102BE3
:04020F00038345829E
:040210000D90F04C11
:0402110006832547F4
:04021200008A4063BB
:040213003E98C060F1
:0402140033B2852557
:040215000C83D0A5E1
:04021600198350A553
:040217003EB2856608
:040218000A83E0C6AF
:040219001F8360C619
:04021A002A9410AB67
:04021B002B9410CC44
:04021C002E9420A953
:04021D001A94F0CA75
:04021E002E8A108193
:04021F00048A2062CB
:040220001FB221EFF9
:0402210016B300E42C
:040222000CD20000FA
:040223000CD20000F9
:040224000B900080BB
:0402250000000000D5
:040226001CA6D246FA
:040227003BB240C6E0
:040228000FAA6306B0
:04022900119E00071B
:04022A0003947021A8
:04022B002494704265
:04022C001382D32145
:04022D002B94D3AA91
:04022E000AC6180FD5
:04022F0027B2340DB1
:040230003E82D1EF4A
:0402310010B2D4082B
:040232000F8A11011D
:0402330034822342AC
:040234000ED2000DD9
:0402350035F2000D91
:040236003C88D040F0
:040237003B044CE94F
:040238000ED2000DD5
:0402390035F2000D8D
:04023A003C8821A03B
:04023B001A044D69EB
:04023C000DC60228C1
:04023D002C94136189
:04023E00069423827D
:04023F003782D10130
:040240003182D10234
:0402410038B7B021F9
:040242001FB7B042F0
:0402430037A6126167
:040244001BA62222B1
:040245001AB270C6B3
:0402460007AA60465D
:040247001CB2D0C64F
:0402480026AA60265C
:0402490006C601A143
:04024A00098A1621E6
:04024B001804494109
:04024C0000000000AE
:04024D0000000000AD
:04024E0000000000AC
:04024F001C2060000F
:040250003F406504C2
:040251003F406504C1
:04025200070421AFCD
:0402530000000000A7
:0402540000000000A6
:0402550000000000A5
:0402560000000000A4
:0402570000000000A3
:0402580000000000A2
:0402590000000000A1
:04025A0000000000A0
:04025B00000000009F
:04025C00000000009E
:04025D00000000009D
:04025E0003C60201D0
:04025F00098A1621D1
:0402600010044BE15A
:0402610033C207217C
:0402620010821621CF
:040263002A281C0920
:040264001BC203E6D0
:040265003D04492FDC
:040266000000000094
:040267000000000093
:040268000000000092
:040269000000000091
:04026A000000000090
:04026B00000000008F
:04026C00000000008E
:04026D00000000008D
:04026E00000000008C
:04026F001F044C2FED
:04027000000000008A
:040271003E1000F04B
:040272002EC6000094
:040273000050000334
:040274002A280046EE
:040275000000000085
:040276000000000084
:040277000050000330
:040278001BC6092177
:040279000DC600A20C
:04027A001F82266356
:04027B0033C6840FF3
:04027C003A242020E0
:04027D002DC6000684
:04027E000EC60007A1
:04027F0015044FF71C
:04028000177A0504E0
:0402810013AB9084A7
:040282002682652645
:0402830032B3054449
:040284003782262275
:040285003A242020D7
:0402860013827087E8
:040287001688206055
:0402880032044FF8F5
:040289001DC200D5BD
:04028A00210C000043
:04028B003E1000F031
:04028C00000000006E
:04028D00000000006D
:04028E00000000006C
:04028F0037C200F57D
:04029000210C00003D
:0402910004C600207F
:040292000050000315
:040293002A280046CF
:040294000000000066
:040295002DC600066C
:040296000EC6000789
:040297000000000063
:040298000000000062
:040299000000000061
:04029A0003C603E1B3
:04029B0009B3D7408C
:04029C003BA610006D
:04029D000388600072
:04029E003C0456F8CE
:04029F002CB38741B4
:0402A0001B88702027
:0402A1003C0456F8CB
:0402A20023C600E08F
:0402A3002EA607403C
:0402A40010AE000098
:0402A500277200E7D5
:0402A60003720021BE
:0402A7002EC870FFEE
:0402A8003904555868
:0402A9002CC61FE759
:0402AA0009C810FF70
:0402AB00340455B80A
:0402AC002FC61FE159
:0402AD0013B280E721
:0402AE0037AA7027D4
:0402AF0013B280E71F
:0402B00019AA70C651
:0402B1001AB280C637
:0402B2002FC61FE153
:0402B3003FA617410A
:0402B4003EAA10C688
:0402B5001A0449EFEF
:0402B6000000000044
:0402B7000AC600C6AD
:0402B8003C8A6626F0
:0402B90031045701B4
:0402BA001BC203E67A
:0402BB001A0449EFE9
:0404000004C600200E
:0404010000500003A4
:040402002A2800465E
:0404030007C6338F66
:04040400347A01EF56
:040405001BC7A0026F
:0404060004AAF04F05
:040407003D7A07C271
:0404080012B1D0401D
:040409002304B0B068
:04040A002DA4266097
:04040B0008049EF152
:04040C00055000FF98
:04040D0028C7FFE01D
:04040E0009A60780B4
:04040F0033B24015AF
:040410002804828FAB
:0404110000000000E7
:0404120000000000E6
:0404130000000000E5
:040414001FC207A15B
:040415000AC8100001
:0404160008049EF147
:0404170028B1A3C0A5
:040418003D048FE030
:040419003E1000F0A1
:04041A0008B203C859
:04041B0037B3F108FA
:04041C001BA686682D
:04041D000E048551F3
:04041E001AC60FE902
:04041F0008C8800287
:040420002A048441E5
:0404210028C61FE9E1
:040422002BC8800360
:04042300270484A185
:040424000FC67FE997
:040425000AA6978903
:040426003CC890013D
:0404270027048541E0
:0404280023C603E6FE
:040429001704888F9D
:04042A001AC20628C4
:04042B003DC7300990
:04042C000CC601EA0F
:04042D003CC207A026
:04042E0007C60026D7
:04042F001FC8000FD3
:040430002F0486F817
:04043100158A0140E7
:040432000FB2F0C64F
:040433001FC8000FCF
:040434002F0486F813
:04043500158A0140E3
:040436000FB2F0C64B
:040437002E7200C65B
:040438001D8A662A89
:0404390034C20606BD
:04043A000AE20120B1
:04043B000AE20120B0
:04043C000ABE0000F4
:04043D000FA60140C5
:04043E001604881107
:04043F0001AA6106A7
:040440002382964934
:0404410013B21108D9
:0404420007C8802047
:0404430029048741C0
:0404440009B250C6E3
:040445003BC980002F
:0404460013048A51C0
:040447002EC601E0DC
:0404480009C990004E
:0404490013048961AE
:04044A003DB3F000CE
:04044B001AC20401CC
:04044C0023C81010A1
:04044D003B048A10D2
:04044E001FB2400099
:04044F000F8A168179
:0404500038721000EE
:040451000CAA00C62B
:040452001DC200D5F2
:04045300210C000078
:040454003E1000F066
:040455002EAA6286E3
:0404560004AA62A6EC
:0404570025AA62C6AA
:040458000FAA62E69F
:040459002DB3B0C649
:04045A000EC60007C3
:04045B002DB1F0C00F
:04045C002686760773
:04045D001FB1E0C02B
:04045E002686760771
:04045F003EB1D0C01A
:04046000268676076F
:040461000CB1C0C05A
:04046200268676076D
:0404630019B1B0C05B
:04046400268676076B
:040465000000000093
:040466000000000092
:0404670037C200F5A3
:04046800210C000063
:04046900000000008F
:04046A00000000008E
:04046B00000000008D
:04046C00000000008C
:04046D001DC200D5D7
:04046E0038C6ABA938
:04046F001C0495AF25
:040470002EB1F3C0F6
:0404710011048E8064
:040472002DC8700021
:04047300310495B10A
:040474000F20B000A5
:0404750027BE00E7B7
:0404760015B2D0E704
:0404770015B2D0E703
:0404780010B3F0E7E6
:040479001CB220C6CB
:04047A000CAA6666FC
:04047B001CB220C6C9
:04047C0019AA70C683
:04047D001C206000DF
:04047E001C0495AF16
:04047F000000000079
:040480000CC603F5AE
:0404810009B193C06A
:040482003B04911096
:0404830038C6ABA923
:040484002EB1F3C0E2
:040485003B0495A0FF
:040486003DC6A9E9DD
:040487001C0495AF0D
:040488002BB203C9C7
:0404890020C600E6A3
:04048A000AA6612637
:04048B002EC6A509CB
:04048C003AC8600208
:04048D0032049201A2
:04048E0001C6A76993
:04048F003B0492EFA9
:040490001CC860061E
:040491001E04928132
:0404920036C6A84979
:040493003B0492EFA5
:0404940019C8600320
:040495003204946138
:0404960011C6A96979
:040497001EB3F7EDAC
:0404980038C6FFE380
:0404990021A631ADBA
:04049A003EC609232E
:04049B00228231ADDB
:04049C001BC207C3B5
:04049D000AA6322356
:04049E0037B271AD53
:04049F0018AAD06D5A
:0404A00031B221ADA7
:0404A1001EAAD6AD0C
:0404A200180495A104
:0404A3003CC86001F0
:0404A400180495A102
:0404A50007C6A629B7
:0404A60025C605263C
:0404A700312062019D
:0404A80036B27626CC
:0404A900258267C67B
:0404AA001CB220C69A
:0404AB002BAA66A66C
:0404AC0012206200B8
:0404AD0005C6004739
:0404AE0028C6000359
:0404AF002DC6000650
:0404B00019B3F2B5D5
:0404B1003604967007
:0404B2000AC6600610
:0404B3003CC7000E34
:0404B40011C8954F87
:0404B5001004970197
:0404B6002FC6000B42
:0404B7002CC6000D42
:0404B8001FC207A1B7
:0404B90003C6976877
:0404BA001908900F7E
:0404BB002DC6000644
:0404BC0019B3F2B5C9
:0404BD00170497F099
:0404BE000AC6600604
:0404BF000DC7080E4F
:0404C00011C8954F7B
:0404C10021049881F9
:0404C2002FC6000B36
:0404C3002CC6000D36
:0404C4001FC207A1AB
:0404C50032C698E8BB
:0404C6001908900F72
:0404C7002DC6000638
:0404C80019B3F2B5BD
:0404C9002B049970F7
:0404CA000AC66006F8
:0404CB000EC7100E3A
:0404CC0011C8954F6F
:0404CD0003049A0189
:0404CE002FC6000B2A
:0404CF002CC6000D2A
:0404D0001FC207A19F
:0404D10010C69A684F
:0404D2001908900F66
:0404D3002DC600062C
:0404D40019B3F2B5B1
:0404D50004049AF091
:0404D6000AC66006EC
:0404D7003FC7180EF5
:0404D80011C8954F63
:0404D90022049B81DD
:0404DA002FC6000B1E
:0404DB002CC6000D1E
:0404DC001FC207A193
:0404DD0031C69BE8A1
:0404DE001908900F5A
:0404DF002DC6000620
:0404E00019B3F2B5A5
:0404E10009049C70FE
:0404E2000AC66006E0
:0404E3002FC7200EF1
:0404E40011C8954F57
:0404E5002F049D0142
:0404E6002FC6000B12
:0404E7002CC6000D12
:0404E8001FC207A187
:0404E9003CC69D6808
:0404EA001908900F4E
:0404EB00000000000D
:0404EC00000000000C
:0404ED00000000000B
:0404EE00000000000A
:0404EF000000000009
:0404F0000000000008
:0404F1000000000007
:0404F2000000000006
:0404F3000000000005
:0404F4000000000004
:0404F5000000000003
:0404F6000000000002
:0404F7000000000001
:0404F8000000000000
:0404F90000000000FF
:0404FA0000000000FE
:0404FB0000000000FD
:0404FC0000000000FC
:0404FD0000000000FB
:0404FE0000000000FA
:0404FF0000000000F9
:0405000000000000F7
:0405010000000000F6
:0405020000000000F5
:0405030000000000F4
:0405040000000000F3
:0405050000000000F2
:0405060000000000F1
:0405070000000000F0
:0405080000000000EF
:0405090000000000EE
:04050A0000000000ED
:04050B001D7A03E072
:04050C003B20000090
:04050D00383800007A
:04050E002EC60000F5
:04050F003704A1F715
:0405100031280A2361
:040511001304A237F6
:04051200070421AF0A
:0405130000000000E4
:0405140000000000E3
:0405150000000000E2
:0405160000000000E1
:0405170000000000E0
:0405180000000000DF
:0405190000000000DE
:04051A0000000000DD
:04051B0000000000DC
:04051C0000000000DB
:04051D0000000000DA
:04051E0000000000D9
:04051F0000000000D8
:0405200000000000D7
:0405210000000000D6
:0405220000000000D5
:0405230000000000D4
:0405240000000000D3
:0405250000000000D2
:040526003304A1CF2A
:0405270000000000D0
:040528000AC61FE3FD
:0405290025A637C309
:04052A0011B281C5C4
:04052B000AAA30A543
:04052C003DB280A5B7
:04052D000CAA56A519
:04052E0002825625CA
:04052F003782E62EFB
:040530000A04AD0FFD
:040531002CE6404331
:040532002EC67FE56D
:0405330028A630A323
:040534000CE640444D
:040535001DA640A41B
:0405360027B2A084C4
:040537003BAA406338
:040538002FE6404525
:040539002EB2A0A599
:04053A002B04AC8F53
:04053B0028B2A785B6
:04053C002EB2A0A596
:04053D0020AA51A5FA
:04053E000FB260A5F3
:04053F0026823623B7
:040540000AAA50654E
:040541000A04AD0FEC
:0405420028B2A785AF
:040543002EB2A0A58F
:0405440020AA51A5F3
:040545000FB260A5EC
:0405460026823623B0
:040547000AAA506547
:040548003BB220A5FD
:0405490026AA50E5A9
:04054A000A04AD0FE3
:04054B0028B2A785A6
:04054C002EB2A0A586
:04054D0020AA51A5EA
:04054E000A04AD0FDF
:04054F000AEE0003AD
:040550000AEE0003AC
:040551002AEE00048A
:0405520002E201C5FB
:04055300209030685C
:040554001E82B06BE8
:040555001B82D00D28
:040556003890408811
:040557001382B08BD0
:040558001B82D00D25
:04055900209050A8F6
:04055A003982B0AB87
:04055B001B82D00D22
:04055C002D04AC2F8F
:04055D000AEE00039F
:04055E000AEE00039E
:04055F002AEE00047C
:0405600002E201C5ED
:040561002EB2A0A571
:0405620007AA50850F
:040563002C04B03183
:040564002EB2A0A56E
:040565000AAA506529
:040566003BB220A5DF
:0405670026AA50E58B
:04056800054450C036
:040569003E385000C8
:04056A00028A16618A
:04056B0039089008B3
:04056C000FA276273D
:04056D0011C8954FCD
:04056E002F088001D1
:04056F00347A01EFEA
:040570000000000087
:040571002AD2000486
:040572002AD2000485
:040573001382B08BB4
:040574000C38B0008F
:040575000000000082
:040576002AD2000481
:040577002AD2000480
:040578003782D08D69
:040579002B38D0004B
:04057A00000000007D
:04057B002AD200047C
:04057C002AD200047B
:04057D0001864604A9
:04057E000C384000F5
:04057F00347A01EFDA
:040580002B08800FB5
:040581001DC680040F
:0405820007AA5085EF
:040583002B04AC8F0A
:040584000000000073
:040585002AE64040E2
:040586002150000FF1
:040587000BC7FFE1BE
:040588000FA6003585
:040589002DA4266017
:04058A001804A09120
:0406000000000000F6
:0406400023C6068047
:04064100249006A952
:040642002150000F34
:040643002CC6000DB4
:040644003782D02EFB
:040645001F82E00F21
:0406460000000000B0
:0406470000000000AF
:0406480000000000AE
:0406490038F4000081
:04064A002704C95761
:04064B0032E6600033
:04064C003B2000004F
:04064D001688E1E04A
:04064E002604C93085
:04064F0025049EEFF1
:0406E0002228BB6FA2
:0406E1001604DC37E8
:0406E2000128BB6EC2
:0406E3001D04DC779F
:0406E4003504A08FAA
:0406E5000000000011
:040700002AC61FE402
:040701002150000F74
:0407020036ECF0E001
:040703002204E07775
:0407040035E660086E
:0407050030A64100D9
:0407060020B3810596
:0407070018A640A14F
:040708002BB380A5EA
:040709001EA640A246
:04070A000E04E211E6
:04070B002BB380A5E7
:04070C0035A40620EA
:04070D001EC6E248DA
:04070E001D04E8914D
:04070F000204E40FED
:040710001EC6E248D7
:040711001904EC2FAC
:040712000604E257A0
:040713002150000F62
:040714001B28B0E00E
:040715001FB2478048
:0407160002AA0640ED
:040717002150000F5E
:040718000DC61C816D
:040719003C8216A167
:04071A000B04E35792
:04071B00292400206D
:04071C002BC60240A6
:04071D000604E3B734
:04071E003B280A0466
:04071F002304E3EFDD
:040720002FC6000BD5
:0407210020C61FC30C
:0407220028A60060A5
:0407230011C6E4A96E
:040724003004EEEFC0
:0407250010C20003FB
:040726001AC6E50901
:040727003804F12F72
:0407280011C6E549C8
:040729001404F62F8F
:04072A003AC20023AC
:04072B001CC6E5A95A
:04072C003804F12F6D
:04072D0017C6E5E91D
:04072E001404F62F8A
:04072F0033C6E629BE
:040730003004EEEFB4
:0407310023AA0620D1
:0407320010C20003EE
:040733001FC6E6A94E
:040734003804F12F65
:0407350014C6E6E917
:040736001404F62F82
:040737002150000F3E
:0407380008C61E0EC3
:0407390035C6E76971
:04073A003604F32F5F
:04073B00213C30002D
:04073C002E8A2622B9
:04073D001B04E83180
:04073E0009C6E809F7
:04073F003D04F50F71
:040740002B04E72F70
:0407410028C6E86975
:040742001404F04F5C
:040743002B08800FF0
:040744002FC6000BB1
:040745002150000F30
:040746002CC61C2E73
:0407470020C61FC3E6
:0407480028A600607F
:0407490025C6E9696F
:04074A003004EEEF9A
:04074B0010C20003D5
:04074C0023C6E9C90E
:04074D003804F12F4C
:04074E0007C6EA09E7
:04074F001404F62F69
:040750003AC2002386
:0407510026C6EA6965
:040752003804F12F47
:0407530001C6EAA948
:040754001404F62F64
:0407550038F4000074
:040756001B04EAD7BF
:0407570034E6600321
:0407580001C6EB49A2
:040759003804F12F40
:04075A0026C6EB893B
:04075B001404F62F5D
:04075C002E8A262299
:04075D001004EAA1F9
:04075E0026C6EC09B6
:04075F001404F04F3F
:040760002B08800FD3
:0407610003C6004487
:0407620007C60026A0
:040763001DAA40C4C7
:040764003104EC97D9
:04076500005000033D
:040766003728417976
:040767001004ECF797
:04076800005000033A
:040769001428417897
:04076A0001C6ED8A4D
:04076B000204F96F1C
:04076C000AC6EDCA02
:04076D002D04FC8FCC
:04076E0028C6EE09A2
:04076F001404F04F2F
:0407700023C6EE4965
:040771001404F04F2D
:0407720004C6EE8942
:040773001404F04F2B
:040774000FC6EEC9F5
:040775001404F04F29
:040776002B08800FBD
:0407770009C6EF2A96
:040778000C04FB6F03
:0407790002C6EF6A5B
:04077A000204F96F0D
:04077B0025C6EFAAF6
:04077C002504F84F09
:04077D002EC6EFEAAB
:04077E002D04FC8FBB
:04077F0026C6F02A70
:040780000204F96F07
:040781001908900FB4
:0407820020C6F08A13
:040783002504F84F02
:040784002BC6F0CAC6
:040785000C04FB6FF6
:0407860001C6F10AAD
:040787000204F96F00
:040788001908900FAD
:0407890011C2006435
:04078A0026C600E59A
:04078B0033B1808086
:04078C000CC6F1EABC
:04078D000204F8402A
:04078E000204F96FF9
:04078F0028C6F22A5C
:040790000C04FB6FEB
:0407910023C6F26A1F
:040792002D04FC8FA7
:0407930013B2108409
:040794001B8A562541
:040795001404F160F7
:040796000FC6F30A8D
:040797000204F96FF0
:040798001908900F9D
:0407990005C600E4AD
:04079A0028C600036A
:04079B0009C6F3AAEE
:04079C000C04FB6FDF
:04079D0002C6F3EAB3
:04079E000C04FA8FBE
:04079F003EB21063F3
:0407A00009AA30A3CF
:0407A10002C6F46A2E
:0407A2002D04FC8F97
:0407A3000A8A462454
:0407A4001A04F360E0
:0407A5002EC6F4EA7E
:0407A6000204F96FE1
:0407A7001908900F8E
:0407A80025C6F54A23
:0407A9002504F84FDC
:0407AA0002C6F58A04
:0407AB000C04FB6FD0
:0407AC0009C6F5CABB
:0407AD002D04FC8F8C
:0407AE002DC6F60A54
:0407AF000204F96FD8
:0407B0001908900F85
:0407B1000CC6F66A12
:0407B2000204F96FD5
:0407B3002BC6F6AAB1
:0407B4000C04FB6FC7
:0407B50006500000EA
:0407B60022C606440D
:0407B7000AC6F72A4D
:0407B8000C04FA8FA4
:0407B9000A8A46243E
:0407BA000304F8112B
:0407BB002DAA50A56E
:0407BC003704F6E127
:0407BD002DC6F7EA64
:0407BE002D04FC8F7B
:0407BF001908900F76
:0407C0003482B62B9E
:0407C1003504F7AF55
:0407C20000500003E0
:0407C3003BEC317961
:0407C4002C04F89772
:0407C50031E66006B3
:0407C60008C600A7BA
:0407C70038A670C61A
:0407C80000500003DA
:0407C9002428617906
:0407CA000A04FDAF71
:0407CB0000500003D7
:0407CC003BEC317958
:0407CD000B04F9B769
:0407CE0031E66006AA
:0407CF0005C6004714
:0407D00019AA70C62C
:0407D10000500003D1
:0407D20024286179FD
:0407D3000A04FDAF68
:0407D40000500003CE
:0407D5003DEC317A4C
:0407D6002904FAD721
:0407D70037E660059C
:0407D8000CB3E0A5D9
:0407D90001A65625FA
:0407DA000A04FDAF61
:0407DB0000500003C7
:0407DC003BEC317948
:0407DD000504FBB75D
:0407DE0031E660069A
:0407DF0024C6002705
:0407E00019AA70C61C
:0407E10000500003C1
:0407E20024286179ED
:0407E3000A04FDAF58
:0407E40000500003BE
:0407E5003BEC31793F
:0407E6000804FCD730
:0407E70031E6600691
:0407E80029C600C757
:0407E90038A670C6F8
:0407EA0000500003B8
:0407EB0024286179E4
:0407EC000A04FDAF4F
:0407ED0023C6190600
:0407EE003C8A6626B5
:0407EF002F04FDC115
:0407F0003808A00F16
:0407F1000000000004
:040B00003005816FCC
:040B01001AB210A56F
:040B020020AA5625AA
:040B03003D20500041
:040B04002B08700F3B
:040B050029E801C01A
:040B060011B281C5E2
:040B07001D82E06EFD
:040B080001AA5025C9
:040B09003DB270A5E4
:040B0A0005C6020218
:040B0B0020AA504587
:040B0C000AAA50657C
:040B0D001AB210A563
:040B0E003D20500036
:040B0F0001C603EC2C
:040B10000E05621755
:040B110029E801C00E
:040B120037E660055D
:040B13002BA6518537
:040B1400098A162113
:040B1500290560311D
:040B16001D82E06EEE
:040B1700030562F779
:040B180029E801C007
:040B190014E660047A
:040B1A003AA6418432
:040B1B0027B2508429
:040B1C0007AA50854F
:040B1D00098A16210A
:040B1E002905603114
:040B1F001D82E06EE5
:040B20002F05641722
:040B210029E801C0FE
:040B220014E6600471
:040B23003AA6418429
:040B240027B2A084D0
:040B250007AA508546
:040B2600098A162101
:040B2700290560310B
:040B28001D82E06EDC
:040B2900080565371F
:040B2A0029E801C0F5
:040B2B0014E6600468
:040B2C003AA6418420
:040B2D0021B2F0847D
:040B2E0007AA50853D
:040B2F00098A1621F8
:040B30002905603102
:040B31001D82E06ED3
:040B32002A056657D3
:040B330029E801C0EC
:040B340014E660045F
:040B35003AA6418417
:040B360021B2F08474
:040B370027B250840D
:040B380007AA508533
:040B3900098A1621EE
:040B3A0029056031F8
:040B3B001D82E06EC9
:040B3C0000056797B2
:040B3D0029E801C0E2
:040B3E0014E6600455
:040B3F0021B2F0846B
:040B400027B2A084B4
:040B410007AA50852A
:040B4200098A1621E5
:040B430029056031EF
:040B44001D82E06EC0
:040B45001AB210A52B
:040B460020AA562566
:040B47003D205000FD
:040B48002005620F13
:040B490011B281C59F
:040B4A0038F400007B
:040B4B0001AA502586
:040B4C003DB280A591
:040B4D0022C6054275
:040B4E0020AA504544
:040B4F003D205000F5
:040B50002EC607ECBA
:040B510015056A37E5
:040B520038F4000073
:040B530037E660051C
:040B54002BA65185F6
:040B5500098A1621D2
:040B560029056031DC
:040B570032056AF702
:040B580038F400006D
:040B590014E660043A
:040B5A003AA64184F2
:040B5B0006B26084FA
:040B5C0007AA50850F
:040B5D00098A1621CA
:040B5E0029056031D4
:040B5F003F056BF7EC
:040B600038F4000065
:040B610014E6600432
:040B62003AA64184EA
:040B630000B2C08498
:040B640007AA508507
:040B6500098A1621C2
:040B660029056031CC
:040B670013056CF70F
:040B680038F400005D
:040B690014E660042A
:040B6A003AA64184E2
:040B6B0000B2C08490
:040B6C0006B26084E9
:040B6D0007AA5085FE
:040B6E00098A1621B9
:040B6F0029056031C3
:040B700010056E17E7
:040B710038F4000054
:040B720014E6600421
:040B730000B2C08488
:040B740000B2C08487
:040B750007AA5085F6
:040B7600098A1621B1
:040B770029056031BB
:040B78001AB210A5F8
:040B790020AA562533
:040B7A003D205000CA
:040B7B003B056A2F9D
:040B7C0011B281C56C
:040B7D0038F4000048
:040B7E0001AA502553
:040B7F003DB280A55E
:040B800021C6064242
:040B810020AA504511
:040B82003D205000C2
:040B83001FC60FEC8E
:040B84001E05709743
:040B850038F4000040
:040B860037E66005E9
:040B87002BA65185C3
:040B8800098A16219F
:040B890029056031A9
:040B8A003405715766
:040B8B0038F400003A
:040B8C0014E6600407
:040B8D003AA64184BF
:040B8E0034B2708489
:040B8F0007AA5085DC
:040B9000098A162197
:040B910029056031A1
:040B9200370572575A
:040B930038F4000032
:040B940014E66004FF
:040B95003AA64184B7
:040B960013B2E08432
:040B970007AA5085D4
:040B9800098A16218F
:040B99002905603199
:040B9A003A0573574E
:040B9B0038F400002A
:040B9C0014E66004F7
:040B9D0013B2E0842B
:040B9E0034B2708479
:040B9F0007AA5085CC
:040BA000098A162187
:040BA1002905603191
:040BA2001AB210A5CE
:040BA30020AA562509
:040BA4003D205000A0
:040BA5003005708F18
:040BA60011B281C542
:040BA70038F400001E
:040BA80001AA502529
:040BA9003DB280A534
:040BAA003CC60942FA
:040BAB0020AA5045E7
:040BAC003D20500098
:040BAD000AC67FEC09
:040BAE00370575D7BB
:040BAF0038F4000016
:040BB00037E66005BF
:040BB1002BA6518599
:040BB200098A162175
:040BB300290560317F
:040BB4003F057697EC
:040BB50038F4000010
:040BB60014E66004DD
:040BB7003AA6418495
:040BB80027B2A0843C
:040BB90007AA5085B2
:040BBA00098A16216D
:040BBB002905603177
:040BBC0032057797F0
:040BBD0038F4000008
:040BBE0014E66004D5
:040BBF0027B2A08435
:040BC00027B2A08434
:040BC10007AA5085AA
:040BC200098A162165
:040BC300290560316F
:040BC4001AB210A5AC
:040BC50020AA5625E7
:040BC6003D2050007E
:040BC700190575CFC8
:040BC80011B281C520
:040BC90038F40000FC
:040BCA0001AA502507
:040BCB003DB280A512
:040BCC0010C60E42FF
:040BCD0020AA5045C5
:040BCE003D20500076
:040BCF0026500007A5
:040BD00009C7FFEC66
:040BD10027057A3743
:040BD20038F40000F3
:040BD30037E660059C
:040BD4002BA6518576
:040BD500098A162152
:040BD600290560315C
:040BD70000057AF7A4
:040BD80038F40000ED
:040BD90014E66004BA
:040BDA0021B2F084D0
:040BDB0007AA508590
:040BDC00098A16214B
:040BDD002905603155
:040BDE001AB210A592
:040BDF0020AA5625CD
:040BE0003D20500064
:040BE10009057A2F59
:040BE20011B281C506
:040BE30001AA5025EE
:040BE4003DB280A5F9
:040BE50022C61E42C4
:040BE60020AA5045AC
:040BE7003D2050005D
:040BE80038F40000DD
:040BE9000B057D3744
:040BEA0014E66004A9
:040BEB0013B21084AD
:040BEC0031AA4624C0
:040BED000F20400095
:040BEE00098A162139
:040BEF000B057D0174
:040BF0002B08700F4F
:040BF10029E801C02E
:040BF2003C7A01C583
:040BF3002150000F7E
:040BF4000DC7FFE248
:040BF50024057EB79E
:040BF60014E660049D
:040BF70010A64044C0
:040BF80007AA508573
:040BF9003BB220A546
:040BFA0020AA5625B2
:040BFB003D20500049
:040BFC002B08700F43
:040BFD0029E801C022
:040BFE003C7A01C577
:040BFF002150000F72
:040C00000DC7FFE23B
:040C0100180580371B
:040C020014E6600490
:040C030030A6404394
:040C04000AAA506583
:040C05003BB220A539
:040C06002BAA56655A
:040C07003D2050003C
:040C080031AA4624A3
:040C09000F20400078
:040C0A002B08700F34
:040C0B003EC6C80019
:040C0C0016200201AB
:040C0D002EC60000EF
:040C0E00352002008B
:040C0F00005000038E
:040C100008C6028E82
:040C11002CC600618C
:040C12002FC78287DF
:040C13002005790F30
:040C14000050000389
:040C150010C6084EAF
:040C16000BC60141C7
:040C170024C7832744
:040C18003805692F03
:040C19000050000384
:040C1A0029C602EEF7
:040C1B002AC600C124
:040C1C0002C60023E9
:040C1D0003C783E79F
:040C1E00280560AF96
:040C1F00005000037E
:040C200039C6200EA3
:040C21003CC60801C4
:040C22000EC78487EE
:040C23003805692FF8
:040C24000050000379
:040C25002AC6000ECD
:040C260003C60201FE
:040C270005C7852751
:040C28001F056F8FA6
:040C29000050000374
:040C2A0005C6040EE9
:040C2B002CC6006172
:040C2C0008C785C7A9
:040C2D00140574CF67
:040C2E00005000036F
:040C2F0008C6050EE0
:040C30002CC600616D
:040C31000DC78667FE
:040C32002005790F11
:040C3300005000036A
:040C34000BC6060ED7
:040C35002CC6006168
:040C360021C7870744
:040C3700140574CF5D
:040C38000050000365
:040C390006C6070ED6
:040C3A000BC600A144
:040C3B0027C787A799
:040C3C00140574CF58
:040C3D000050000360
:040C3E001BC6080EBB
:040C3F0006C60041A4
:040C400037C78847E3
:040C41002005790F02
:040C4200005000035B
:040C430015C60A0EBA
:040C44001BC788C77B
:040C450007057FAF71
:040C46000050000357
:040C47003FC60A2E6C
:040C480006C600419B
:040C490002C60023BC
:040C4A001DC78987B2
:040C4B00280560AF69
:040C4C000050000351
:040C4D0034C60A6E31
:040C4E0032C78A0718
:040C4F0007057FAF67
:040C5000005000034D
:040C510039C60A8E08
:040C520006C6004191
:040C530002C60023B2
:040C540015C78AC76F
:040C5500280560AF5F
:040C56000050000347
:040C57000BC62B0E8F
:040C580021C6008130
:040C59001EC78B67C0
:040C5A00140574CF3A
:040C5B000050000342
:040C5C000DC62BAEE8
:040C5D002CC6006140
:040C5E0013C78C0725
:040C5F00140574CF35
:040C6000005000033D
:040C61000DC62C2E62
:040C62002CC600613B
:040C630002C60023A2
:040C640034C78CC73E
:040C6500280560AF4F
:040C66000050000337
:040C670021C62CAEC8
:040C680006C600417B
:040C69003FC78D678D
:040C6A002005790FD9
:040C6B000050000332
:040C6C0029C62E0E59
:040C6D0006C6004176
:040C6E001DC78E0709
:040C6F00140574CF25
:040C7000005000032D
:040C710022C62E4E1B
:040C720031C78E8771
:040C730007057FAF43
:040C74000050000329
:040C750024C62F0E54
:040C760006C600416D
:040C770002C600238E
:040C78001BC78F47C0
:040C7900280560AF3B
:040C7A0029E64046E1
:040C7B000E058F775C
:040C7C002150000FF4
:040C7D0009C61E0581
:040C7E002E8256A5C7
:040C7F00222460A02B
:040C800025049EEFBA
:040D00002150000F6F
:040D010029C7FFEB14
:040D020015A6B70E6D
:040D03003EC201CD1E
:040D040038F40000BF
:040D050004C603E934
:040D06002EC61FEAEC
:040D07002C05A0F720
:040D080032E660006F
:040D090038F40000BA
:040D0A003DB3F00005
:040D0B002605A750C2
:040D0C0039B3900166
:040D0D0006A6A02175
:040D0E001505A8B16E
:040D0F002AB3E00221
:040D100000A6904267
:040D110037822622DD
:040D12000FA60663BF
:040D13000FB310000A
:040D14000CC8200FD8
:040D15002705A431D9
:040D160009C8200ADE
:040D17002705A431D7
:040D18002EC82005BC
:040D19002705A431D5
:040D1A0025C8201FA9
:040D1B000305A61115
:040D1C0028C82006BD
:040D1D002705A431D1
:040D1E000BC82007D7
:040D1F002705A431CF
:040D20003805A8AF3B
:040D21003EAE0042A0
:040D220024C60011D2
:040D230037822231C0
:040D24002405A542BB
:040D250038F400009E
:040D260014E660046B
:040D270037B3F0846A
:040D28002AC603F1E3
:040D290037822231BA
:040D2A00372440002A
:040D2B002B820060B7
:040D2C00137220849A
:040D2D00098A1621F8
:040D2E000505A461B2
:040D2F000205A0EF2A
:040D300030B3F6ECFA
:040D310038F4000092
:040D320014E660045F
:040D330037B3F0845E
:040D34002C05A6974D
:040D3500372440001F
:040D36002B820060AC
:040D3700098A1621EE
:040D38000005A621EB
:040D39000205A0EF20
:040D3A001EB3F001F3
:040D3B0034A6116168
:040D3C003305A820B3
:040D3D0038F4000086
:040D3E0014E6600453
:040D3F001DA646C4E3
:040D400015AA40218F
:040D41003BB3500070
:040D42003BB3A0001F
:040D43003124100047
:040D44000205A0EF15
:040D45002E8AE62EDE
:040D46001C05AA8F4F
:040D47001FB2478010
:040D480028AA06606F
:040D49002150000F26
:040D4A000DC61C8135
:040D4B003C8216A12F
:040D4C003105A9972D
:040D4D002924002035
:040D4E002BC602406E
:040D4F001005A9F7EB
:040D50003B280A042E
:040D51003405AA3784
:040D52003B05AA4F64
:040D5300000000009C
:040D540019C201C2FD
:040D550019C201AE10
:040D560038F400006D
:040D570019C206E1D6
:040D580026504C11C4
:040D590026C7B6E310
:040D5A001805AB5776
:040D5B0004C60405C1
:040D5C0032E660001B
:040D5D0038F4000066
:040D5E003DB3F000B1
:040D5F0009861021D0
:040D60003D05AC4061
:040D610001A210617A
:040D62001B8A56256D
:040D63001E05ABC1FD
:040D64001D88E040C6
:040D65001505AB784D
:040D66000CA216E1E4
:040D670032E6600010
:040D680016881000D9
:040D6900323C100008
:040D6A003305A8EFB6
:040D6B000000000084
:040D6C002150000F03
:040D6D0029C7FFEBA8
:040D6E0015A6B70E01
:040D6F0004C603E9CA
:040D70002EC61FEA82
:040D71001B05AE3779
:040D720038F4000051
:040D73001005AE7742
:040D740032E6600003
:040D75003DB3F0009A
:040D76001F05B6F0AF
:040D770039B39001FB
:040D780006A6A0210A
:040D79000B05B9D1DC
:040D7A002AB3E002B6
:040D7B0000A69042FC
:040D7C003782262272
:040D7D000FA6066354
:040D7E000FB310009F
:040D7F000CC8200F6D
:040D80003105B191F7
:040D810009C8200A73
:040D82003105B191F5
:040D83002EC8200551
:040D84003105B191F3
:040D850025C8201F3E
:040D86001E05B59100
:040D870028C8200652
:040D88003105B191EF
:040D89000BC820076C
:040D8A003105B191ED
:040D8B002605B9CFB1
:040D8C003372262C6C
:040D8D00188AC62CCE
:040D8E0029C600086A
:040D8F002BC600056A
:040D90001D05B21774
:040D910003E8000073
:040D92002B82006050
:040D930010B3F107A1
:040D94003105B297DC
:040D950014E66004FC
:040D96003AA64184B4
:040D97000AC8800FF7
:040D98001E05B488F8
:040D990015728084CB
:040D9A001FAA40A5A7
:040D9B00098A16218A
:040D9C003205B51156
:040D9D0013828048F5
:040D9E0005C8801BE9
:040D9F003D05B2104C
:040DA0001AB210A5CE
:040DA10020AA562509
:040DA200063C5000BB
:040DA3001705B1CFB0
:040DA40015727084D0
:040DA5002B8A80E72E
:040DA60015727084CE
:040DA7003505B34F0C
:040DA8001AB210A5C6
:040DA90020AA562501
:040DAA00063C5000B3
:040DAB003505AE2F2D
:040DAC001D05B597D5
:040DAD0003E8000057
:040DAE002B82006034
:040DAF003C05B5F753
:040DB00014E66004E1
:040DB10013B21084E5
:040DB20031AA4624F8
:040DB300343C40008C
:040DB400098A162171
:040DB5003705B581C8
:040DB6003505AE2F22
:040DB70018B350011C
:040DB80032B3A02191
:040DB9001505B7372E
:040DBA0029E8002004
:040DBB0004A6062361
:040DBC002E8AE62E67
:040DBD003905B7B786
:040DBE0014E66004D3
:040DBF0036B2E02543
:040DC0003BB220A57D
:040DC10034A64162B1
:040DC20020AA5045CE
:040DC3001AB210A5AB
:040DC4000AAA5065C2
:040DC5001AB210A5A9
:040DC60020AA5625E4
:040DC700063C500096
:040DC80025A6362303
:040DC9001805AE312A
:040DCA0012AA4625FE
:040DCB000E05B977E1
:040DCC00063C500091
:040DCD003505AE2F0B
:040DCE000000000021
:040DCF001FB2478088
:040DD00028AA0660E7
:040DD1002150000F9E
:040DD2000DC61C81AD
:040DD3003C8216A1A7
:040DD4000005BA97C5
:040DD50029240020AD
:040DD6002BC60240E6
:040DD7002105BAF741
:040DD8003B280A04A6
:040DD9000B05BB3714
:040DDA000405BB4F02
:040DDB000000000014
:040E00001BC20760AA
:040E01002150000F6D
:040E02000BC7FFE13A
:040E030001A6002A1A
:040E04003405C811D8
:040E0500137A00005C
:040E060022A6002BF5
:040E07003405C811D5
:040E08000EC67FE2B1
:040E090007B2C04329
:040E0A003FAA206279
:040E0B000750000B81
:040E0C000CC7FFE927
:040E0D0031C20740A7
:040E0E0013C620E106
:040E0F0002A6002C0B
:040E10003405C811CC
:040E11002AC7CA48DA
:040E12002EB01000EE
:040E13002005C38073
:040E1400137A00004D
:040E15002EC7FFE302
:040E16002EA63003D1
:040E170011C20064A0
:040E18000DC6000102
:040E19001EC6400EA3
:040E1A0006C7CD48F2
:040E1B000705C40FF4
:040E1C00137A000045
:040E1D0021A6002DDD
:040E1E002A05C411CC
:040E1F0008C7C8C870
:040E20001A2C000088
:040E210014C7C680AC
:040E220004C60405F9
:040E2300049056AD34
:040E240011C760E6AC
:040E2500288260A619
:040E2600242400C0C0
:040E270036C761C6A3
:040E2800288260A616
:040E29001AC610A035
:040E2A0000000000C4
:040E2B0000000000C3
:040E2C0000000000C2
:040E2D0000000000C1
:040E2E0000000000C0
:040E2F0000000000BF
:040E30002705C617B5
:040E3100242400C0B5
:040E3200213000006B
:040E33002805C66F59
:040E340009C6000FDC
:040E350000000000B9
:040E36001F389000D1
:040E370000000000B7
:040E38003E38A000A0
:040E390000000000B5
:040E3A000C38B000C0
:040E3B0000000000B3
:040E3C001938C000A1
:040E3D0000000000B1
:040E3E002B38D0007D
:040E3F002B08800FED
:040E40002EC60000BA
:040E410021C7446120
:040E4200098A1621E2
:040E4300292400203E
:040E44003505C88F19
:040E450000000000A9
:040E46000CE2018039
:040E470026E201A0FE
:040E480005E201A11D
:040E490003B2C0210F
:040E4A0002AA0020D8
:040E4B0002A60040BB
:040E4C000524014038
:040E4D002582A62A2A
:040E4E000AA6A12A25
:040E4F002D8AB62B07
:040E50000C0880000A
:040E51003605D08F03
:040E52000CE201802D
:040E53000CE201802C
:040E5400000000009A
:040E55000000000099
:040E56000000000098
:040E57000000000097
:040E58000000000096
:040E59000000000095
:040E5A000000000094
:040E5B000000000093
:040E5C000000000092
:040E5D000000000091
:040E5E002FE20181FD
:040E5F002FE20181FC
:040E600003B2C021F8
:040E61001AAA1000B9
:040E620002A60040A4
:040E63000524014021
:040E64002582A62A13
:040E65000AA6A12A0E
:040E66002D8AB62BF0
:040E67000000000087
:040E68000C088000F2
:040E69003605D08FEB
:040E6A000CE2018015
:040E6B000CE2018014
:040E6C0002A600409A
:040E6D001BA201C003
:040E6E0003820021DA
:040E6F000A8A462481
:040E70001305CEB1E7
:040E7100000000007D
:040E7200000000007C
:040E7300000000007B
:040E74002B08800FB8
:040E750037241140CD
:040E76002582A62A01
:040E77000AA6A12AFC
:040E78002D8AB62BDE
:040E79003805D090D8
:040E7A000CE2018005
:040E7B000CE2018004
:040E7C0002A600408A
:040E7D0038A201C1D5
:040E7E0011C2006439
:040E7F000A8A462471
:040E80001305CEB1D7
:040E8100000000006D
:040E8200000000006C
:040E83002B08800FA9
:040E84003E38A00054
:040E85000000000069
:040E86000C38B00074
:040E87001A2C000021
:040E88000BC600A1F4
:040E89001305D13745
:040E8A00162410C05A
:040E8B003EC682409D
:040E8C001505D197E0
:040E8D003B280A04F0
:040E8E00070421AF85
:040E8F00000000005F
:040FFE003E04018F1D
:040FFF003E04018F1C
:00000001ff
